:020000040000FA
:06000000D8EF00F0120031
:06002A000100E8010000E6
:08003000800000000D0000003B
:0C004400D9CFE6FFE1CFD9FF040EE12682
:10005000DF6A010EDB6A020EDB6A030EDB6AE00E6A
:10006000926E936E800E956ED70EC16E8068816819
:10007000010EDB50EA6A800FE96E000EEA22EF50B3
:10008000836E050EDF5C02E280900CD0050EDF5C13
:10009000036E010E035204E0E846FE0B0306FCE18A
:1000A000E81C816EDF2ADF5002081CE2DF6A030EC3
:1000B000DBCFF3FFDB2AF35006080DE2020EDB2A4A
:1000C000DBCF03F000018C51D880035402E2020E12
:1000D000DB6A030EDB6A020EDB50E76E010EE7CF30
:1000E000DBFF0BD0010EDB2ADBCF03F000018C51CC
:1000F000D880035402E2010EDB6A3E0EE66EE6ECA7
:1001000000F0E552B3D7D9CFE1FFE552E7CFD9FFF1
:020110001200DB
:0E0112002A0EF66E000EF76E000EF86E00015B
:100120000900F550926F0900F550936F03E1926753
:1001300001D03DD00900F5508D6F0900F5508E6F4C
:100140000900F5508F6F09000900F550E96E0900AC
:10015000F550EA6E090009000900F550906F09009A
:10016000F550916F09000900F6CF94F0F7CF95F0A4
:10017000F8CF96F08DC0F6FF8EC0F7FF8FC0F8FF66
:100180000001905302E1915307E00900F550EE6E33
:100190009007F8E29107F9D794C0F6FF95C0F7FFF2
:1001A00096C0F8FF00019207000E935BBFD71200C4
:1001B00015EE00F025EE00F0F86A019CA68EA69CD4
:0C01C00089EC00F022EC00F0FDD71200EA
:0401CC00FF0EE350EF
:1001D000026E1B0E00D001D0200EE76EE72EFED778
:0801E000022EFAD700D0120034
:0801E8000103070F1F3F7F3FD9
:0501F0001F0F07030BC7
:00000001FF
